:020000040000FA
:040000006D303A28FD
:08000800A000030EA100831209
:1000100005191028831601178312B23081002B288E
:1000200083160113831203140B190310A80DA90DD5
:10003000AA0DAB0DAC0DAC16FF302C02031D2B2806
:10004000FA302B02031D2B2831152A08AF0029088E
:10005000AE002808AD008B100B11210E8300A00EFE
:04006000200E090065
:0C007400203084008001840A6030040207
:10008000031C3C281230B00097218316FF239000F8
:10009000831283160C308505870183128501870141
:1000A000073099000030831691008312C830831600
:1000B0008100831231309000003083168C0083124F
:1000C00010308B00831600309B001C141A0883121A
:1000D000BC00851DDB21831610309B001C141A0800
:1000E0008312BD00D32181018E018F010B118B1072
:1000F0000B108C018B178A2031198D20B30B8828A7
:10010000031085190314B90DF030390203191221B7
:1001100000227B2864003210080031110130B70042
:100120008B132030370783169B001C141A08831288
:10013000A4001030370783169B001C141A08831282
:10014000A300A6000230A6060030370783169B00E6
:100150001C141A088312A200A7000130A7068B17EF
:10016000321CB82822090339A200A309A409A50951
:1001700024082F02031D0C2923082E02031D0C291D
:1001800022082D02031D0C2901303702031DCD2842
:100190003D18CD283D143E14A22102303702031D24
:1001A000D628BD18D628BD143E14A421033037022A
:1001B000031DDF283D19DF283D153E14A62104301C
:1001C0003702031DE828BD19E828BD153E14A821F3
:1001D00005303702031DF1283D1AF1283D163E1463
:1001E000AA2106303702031DFA28BD1AFA28BD16C7
:1001F0003E14AC2107303702031D03293D1B0329A0
:100200003D173E14AE2108303702031D0C29BD1BDB
:100210000C29BD173E14B021B70A09303702031864
:10022000080090280130B600B300B400B500B70054
:1002300085018701B1138A20B30B4A290310851960
:100240000314B90DF030390203197129B40B4A298E
:10025000013037020319BB21023037020319BE21D6
:10026000033037020319C121043037020319C421B6
:10027000053037020319C721063037020319CA2196
:10028000073037020319CD21083037020319D02176
:100290009630B400311D1B293111321C54292D090F
:1002A0000339AD00AE09AF092F1C1B298E018F0148
:1002B0000C1C1B290C102E1E1B298B1320303707FA
:1002C000BB002F08BA00842110303707BB002E086E
:1002D000BA00842100303707BB002D08BA00842102
:1002E0008B1785018701B70AB60109303702031C55
:1002F0001B29D32108003E1C08003E101030BB0013
:100300003D08BA00842108008B133A0883161C1597
:100310009A003B089B0055309D00AA309D009C141C
:1003200064009C1890291C1183128B170800FF3061
:10033000D000D415D515D615D715D915DA15DB1576
:10034000DC150800F130B329F230B329F430B329B9
:10035000F830B3291F30B7292F30B7294F30B729CC
:100360008F30B7290800BD050F30D2040800BD0545
:10037000F030D204080010308506080020308506D1
:100380000800213085060800223085060800183054
:100390008706080021308706080009308706080014
:1003A0002930870608003D08D200031D08001130DF
:1003B000BD00D2000800B601B301B4013C1CE32922
:1003C000BC01BC14E529BC013C143C08B600640027
:1003D000E929EA29EB29EC29ED29B41B0516B41FFC
:1003E0000512B30BE729B40BE7290310B60CB608C6
:1003F000031DE7290030BB003C08BA008421080037
:100400008F08031908008F01D00F1A2BD00A0E3065
:100410005205031D1A2A541D102AD4015416282AE5
:10042000D41D152AD4015416282A541E282AD40172
:10043000D414282AD41C1F2AD4015415282A541D48
:10044000242AD401D415282A541E282AD40154154C
:1004500001305205031D3B2A551D312AD501551681
:10046000492AD51D362AD5015516492A551E492A2D
:10047000D501D514492AD51C402AD5015515492A3C
:10048000551D452AD501D515492A551E492AD5019C
:1004900055150B305205031D5C2A561D522AD601F4
:1004A00056166A2AD61D572AD60156166A2A561E8D
:1004B0006A2AD601D6146A2AD61C612AD601561594
:1004C0006A2A561D662AD601D6156A2A561E6A2A37
:1004D000D601561507305205031D7D2A571D732A74
:1004E000D70157168B2AD71D782AD70157168B2A82
:1004F000571E8B2AD701D7148B2AD71C822AD701E3
:1005000057158B2A571D872AD701D7158B2A571EB7
:100510008B2AD70157151030BC1811305205031D16
:10052000A02A591D962AD9015916AE2AD91D9B2AEF
:10053000D9015916AE2A591EAE2AD901D914AE2AAC
:10054000D91CA52AD9015915AE2A591DAA2AD901A3
:10055000D915AE2A591EAE2AD90159155030BC18EA
:1005600051305205031DC32A5A1DB92ADA015A1601
:10057000D12ADA1DBE2ADA015A16D12A5A1ED12AE8
:10058000DA01DA14D12ADA1CC82ADA015A15D12A7A
:100590005A1DCD2ADA01DA15D12A5A1ED12ADA01DA
:1005A0005A15E030BC18E1305205031DE62A5B1DE8
:1005B000DC2ADB015B16F42ADB1DE12ADB015B167A
:1005C000F42A5B1EF42ADB01DB14F42ADB1CEB2A81
:1005D000DB015B15F42A5B1DF02ADB01DB15F42A35
:1005E0005B1EF42ADB015B152030BC18213052055C
:1005F000031D092B5C1DFF2ADC015C16172BDC1D7B
:10060000042BDC015C16172B5C1E172BDC01DC14A1
:10061000172BDC1C0E2BDC015C15172B5C1D132B20
:10062000DC01DC15172B5C1E172BDC015C157B2114
:100630003D08D2005008D1000C305405031D0512AE
:100640000C305505031D85120C305605031D051091
:100650000C305705031D85100C305905031D07107C
:100660000C305A05031D87120C305B05031D071261
:100670000C305C05031D871151080E020318642B12
:1006800012305405031D051612305505031D85163D
:1006900012305605031D051412305705031D85142D
:1006A00012305905031D071412305A05031D871611
:1006B00012305B05031D071612305C05031D8715FC
:1006C000FF305002031908008F08031D08008A201C
:1006D00051080E02031C642B18305405031D05122B
:1006E00006305405031D051618305505031D8512E7
:1006F00006305505031D851618305605031D0510D7
:1007000006305605031D051418305705031D8510C6
:1007100006305705031D851418305905031D0710B1
:1007200006305905031D071418305A05031D87129A
:1007300006305A05031D871618305B05031D071286
:1007400006305B05031D071618305C05031D871175
:0A07500006305C05031D8715080044
:084000000400030002000600A9
:02400E00CC01E3
:10420000010078007A007C007E007B0079007F004E
:104210007D007A0078007E007C00FF00FF00FF0038
:104220000000F200F600FA00FE00F200F600FA00CC
:10423000FE00F200F600FA00FE00FF00FF00FF00A3
:10424000010005000500050005000900090009003E
:1042500009000D000D000D000D00FF00FF00FF0024
:10426000FF00FF00FF00FF00FF00FF00FF00FF0056
:10427000FF00FF00FF00FF00FF00FF00FF00FF0046
:10428000FF00FF00FF00FF00FF00FF00FF00FF0036
:10429000FF00FF00FF00FF00FF00FF00FF00FF0026
:1042A000FF00FF00FF00FF00FF00FF00FF00FF0016
:1042B000FF00FF00FF00FF00FF00FF00FF00FF0006
:1042C000FF00FF00FF00FF00FF00FF00FF00FF00F6
:1042D000FF00FF00FF00FF00FF00FF00FF00FF00E6
:1042E000FF00FF00FF00FF00FF00FF00FF00FF00D6
:1042F000FF00FF00FF00FF00FF00FF00FF00DD00E8
:00000001FF
